:020000040800F2
:10000000009000208D180008DD140008E11400089D
:1000100000000000000000000000000000000000E0
:10002000000000000000000000000000E5140008CF
:100030000000000000000000E9140008ED140008B2
:10004000DD18000800000000DD180008DD180008B9
:10005000DD180008DD180008F9140008051500086F
:10006000000000001115000821150008DD18000827
:10007000DD180008DD180008DD1800080000000089
:10008000DD180008DD180008DD180008DD1800087C
:10009000DD180008DD180008DD180008DD1800086C
:1000A000DD180008DD180008DD1800083915000803
:0800B000DD180008DD1800084E
:1000B80010B5064C2378002B07D1054B002B02D036
:1000C800044800E000BF0123237010BD2400002075
:1000D8000000000050650008044B10B5002B03D049
:1000E8000349044800E000BF10BDC04600000000FE
:1000F80028000020506500080023C25C0133002A54
:10010800FBD1581E70470000002243088B4274D36D
:1001180003098B425FD3030A8B4244D3030B8B4200
:1001280028D3030C8B420DD3FF22090212BA030C09
:100138008B4202D31212090265D0030B8B4219D3EA
:1001480000E0090AC30B8B4201D3CB03C01A52410A
:10015800830B8B4201D38B03C01A5241430B8B4252
:1001680001D34B03C01A5241030B8B4201D30B033B
:10017800C01A5241C30A8B4201D3CB02C01A524162
:10018800830A8B4201D38B02C01A5241430A8B4225
:1001980001D34B02C01A5241030A8B4201D30B020E
:1001A800C01A5241CDD2C3098B4201D3CB01C01A28
:1001B800524183098B4201D38B01C01A5241430932
:1001C8008B4201D34B01C01A524103098B4201D320
:1001D8000B01C01A5241C3088B4201D3CB00C01A8D
:1001E800524183088B4201D38B00C01A5241430805
:1001F8008B4201D34B00C01A5241411A00D201462A
:10020800524110467047FFE701B5002000F0F0F8B2
:1002180002BDC0460029F7D076E7704703460B4376
:100228007FD4002243088B4274D303098B425FD3E7
:10023800030A8B4244D3030B8B4228D3030C8B4213
:100248000DD3FF22090212BA030C8B4202D31212F9
:10025800090265D0030B8B4219D300E0090AC30BCE
:100268008B4201D3CB03C01A5241830B8B4201D37B
:100278008B03C01A5241430B8B4201D34B03C01A64
:100288005241030B8B4201D30B03C01A5241C30ADC
:100298008B4201D3CB02C01A5241830A8B4201D34D
:1002A8008B02C01A5241430A8B4201D34B02C01A37
:1002B8005241030A8B4201D30B02C01A5241CDD2DC
:1002C800C3098B4201D3CB01C01A524183098B4227
:1002D80001D38B01C01A524143098B4201D34B0110
:1002E800C01A524103098B4201D30B01C01A524173
:1002F800C3088B4201D3CB00C01A524183088B42FA
:1003080001D38B00C01A524143088B4201D34B00E2
:10031800C01A5241411A00D2014652411046704754
:100328005DE0CA0F00D04942031000D34042534059
:1003380000229C4603098B422DD3030A8B4212D319
:10034800FC22890112BA030A8B420CD3890192114B
:100358008B4208D3890192118B4204D389013AD088
:10036800921100E08909C3098B4201D3CB01C01A5D
:10037800524183098B4201D38B01C01A5241430970
:100388008B4201D34B01C01A524103098B4201D35E
:100398000B01C01A5241C3088B4201D3CB00C01ACB
:1003A800524183088B4201D38B00C01A5241D9D2E3
:1003B80043088B4201D34B00C01A5241411A00D264
:1003C8000146634652415B10104601D34042002B60
:1003D80000D54942704763465B1000D3404201B5DF
:1003E800002000F005F802BD0029F8D016E7704794
:1003F8007047C046F0B5DE46454657464E46E0B51E
:1004080087B0009201930B031B0B9B46CA0F4B004E
:10041800040080465B0D029200D16AE1D44A9342FF
:1004280000D18CE15946420FC9000A4380210904D2
:100438001143C2009046CF4A894692469A44002307
:1004480000240393009E019F3B031B0B9B467B00EC
:1004580030005B0DFD0F002B00D128E1C44A934208
:1004680000D177E15946720FC9000A438021090477
:1004780011438B46BF49F2008C4651466344CB1A60
:100488009A460023029E6E400F2C27D8BA49A40032
:1004980009598F46CB464246029E039B022B16D033
:1004A800032B00D1A6E2012B00D0DFE000220023BD
:1004B800002490461B052343F607334340461900A2
:1004C80007B0F0BCBB46B246A946A046F0BD002224
:1004D80000249046A64BEDE72E00DFE7CB4500D27F
:1004E800D4E100D1CFE101235B429C464446484613
:1004F8000027E2445B46150E1B021D43190C2B0412
:10050800120200951D0C914602910395FFF782FE99
:1005180002006A430B04210C804619438A4209D918
:10052800009D0123AC465B4261449C46E0448D42F9
:1005380000D8FBE1881A0299FFF76CFE039A24049D
:1005480042430904240C03000C43A24206D9009933
:10055800013B8C466444A14200D8E1E1A01A42461E
:1005680012041A4393464B4659461B0C1D0004932C
:100578000B0449460904090C0C001B0C5C43120CC3
:100588006B43884651436A43250CAC465B18634469
:10059800994203D9802149028C466244190C2404EB
:1005A8001B04240C8A181C19904202D316D1A742A6
:1005B80014D25B46009D013B4F4405934F459B4138
:1005C800AC465B426344C018854200D3A1E1824235
:1005D80000D9F6E100D1F1E1059B9B463C1BA742FF
:1005E800BF41009D801A7F42C01B854200D1D0E1E7
:1005F8000299FFF70FFE039A0B044243210C0700F0
:1006080019438A4200D978E1881A0299FFF702FE55
:10061800039A240442430904240C03000C43A24215
:1006280000D95DE14146A41A3A041A43049D130413
:100638001B0C594347466B439C46100C47430B0C15
:10064800BC44634468439F4203D980256D02AC468D
:1006580060441F0C09041B04090C3F185B18BC42BA
:1006680000D202E100D1FDE001231A43434B534479
:10067800002B00DCAEE0510700D098E15946C901D3
:1006880006D559463E4B194080238B46DB00534420
:100698003C498B4200DD1AE75946D2084907114305
:1006A8005A465B0554028846240B5B0D02E75A46FE
:1006B800009B1A4300D17EE05B46002B00D100E18D
:1006C800584600F0E3FC020003000B3A1D27009E89
:1006D800BA1A19005846D6400839884032000243F1
:1006E8009346009A8A40284953448A469A440023EC
:1006F800C8E65B460343994656D05B46002B00D1BB
:10070800CDE0584600F0C2FC0B235B429C46020039
:10071800844466461D239B1B260011005846DE4074
:100728000839884033000343994623008B40984694
:10073800164B00249B1A9A460023039382E65A46D6
:10074800024391462AD100229A4602239046082461
:10075800039377E65A46009B1A430D4B9C46E244A6
:10076800002A17D102231C4300239B46023389E643
:10077800FF07000001FCFFFF68650008FF03000099
:10078800FFFFFFFEFE070000F30300000DFCFFFF64
:1007980001F8FFFF032332001C4373E69A46032344
:1007A800D9460C2403934DE6002398469A46013314
:1007B8000424039346E601231C4300239B4601338C
:1007C80060E60023802498460026924B240371E6B5
:1007D800012252420121C91A382900DD66E61F2983
:1007E80000DCABE01F204042C31A5846D840030043
:1007F800202904D058468849514488400243511E54
:100808008A411A43072319000024114013420CD0CF
:100818000F231340042B00D1F9E0111D91429B4195
:100828000A005B4259075B021C0BD2080A43904638
:1008380000233FE680244B462403234209D05B462D
:10084800234206D11C4324032E009046714B240BEF
:1008580030E680244B4624031C432403029E6D4B40
:10086800240B27E6002B00D100E70098511E844690
:100878006444844200D284E0BC4200D2AEE000D19D
:10088800C1E00A00F0E6424500D92CE64B46DC07F9
:10089800580843465B081C434346DF072AE600F036
:1008A800F5FB15239C4684440200634620321C2B2A
:1008B80000DC2EE723000838834099460023984639
:1008C80036E700F0E3FB02000300153220331C2A50
:1008D80000DCFBE600990838814000228B4602E7DD
:1008E8000099013B8C466444A14200D99AE6A24291
:1008F80000D897E6831E644494E6AC466144013F01
:100908008D4200D980E68A4200D87DE6871E614480
:100918007AE6854200D05FE6B94500D95CE656E63E
:10092800A24200D81AE6831E644417E68A4200D819
:1009380000E6AC46831E98466144FBE53748140040
:10094800504482405B4617008340CC407A1E974152
:1009580023433B431A005B46CB40510709D00F2184
:100968001140042905D0111D9142924152429B1811
:100978000A00190200D455E70022012300249046FA
:1009880098E50A00BC4200D06EE64B4500D06BE605
:100998006CE6234B234A5344924500DA18E70121B9
:1009A80049420A1D8A42894149428B4466E60F2121
:1009B8001140042900D161E61100F2E7BC4200D8D9
:1009C8000AE602235B429C4600994F444F459B41EF
:1009D800E3448C465B426344C018FFE54946009DEA
:1009E800480048458941AC46494261448146023A3B
:1009F8006418C7E780245B4624031C4324039046FD
:100A0800044B240B56E59945E8D30A00BDE70023BB
:100A180008E7C046FF0700003E0400001E0400006F
:100A2800FF03000002FCFFFFF0B55746DE464E46C6
:100A38004546E0B51F000B031B0B16009A46CA0F6C
:100A48004B000400934687B05B0D00D1D5E0BB4A4C
:100A5800934200D1F8E05146420FC9000A43802171
:100A680009041143C2009146B54A8A469D180023DD
:100A7800984602933C037B00FA0F3000240B5B0D71
:100A8800009200D196E0AD4A934231D0720FE40053
:100A98002243802424041443A94AF0009446634462
:100AA8005B195A1C0192424600260A2A42DC5A4621
:100AB80000994A4093464246022A32DC013A012A0A
:100AC80000D949E1022E00D1CAE0012E3DD1002310
:100AD8000024002210005A461B052343D207134363
:100AE800190007B0F0BCBB46B246A946A046F0BD07
:100AF800924B2643EB18002E00D1BBE0032241465F
:100B080011435A46884600994A40802109018C467B
:100B180029006144019141460A2900DD33E29346E8
:100B28000326424601279740A6213A00C9000A40F9
:100B38000F4231D0029E022E00D135E2032E00D1A1
:100B4800D2E154464846012EC1D0019A7D4B9446C5
:100B58006344002B00DCC0E0420709D00F220240AA
:100B6800042A05D0021D8242804140422418100008
:100B7800E20106D5744B019A1C4080239446DB00A1
:100B88006344724A93426BDC6207C00864025B05E7
:100B98000243240B5B0D9DE7902189000F4263D12E
:100BA80088223A4200D1D7E0009BA2469B46814664
:100BB8000296BFE72300334300D17FE0002C00D129
:100BC800ADE1200000F062FA020003000B3A1D209C
:100BD8001900821A30000839D0408C400443300094
:100BE80088405B4AEB1A944663445A1C0192424679
:100BF80000260A2A00DC5AE79CE753460343994635
:100C080054D05346002B00D177E1504600F03EFA0D
:100C18000B235B429C46020084441100504608396D
:100C280088401D23804660461B1A2000D8400300D8
:100C3800404603439A4623008B4099460023444D7F
:100C48009846AD1A029315E752460243914626D1BB
:100C580000221D000223924608329046029309E7BB
:100C680000240022354B35E7002380249B462403CB
:100C7800324B2FE70222414611438022120194464B
:100C88002A006244884601920A2900DD52E75A4642
:100C98000020009904004A40934602260BE70C22E4
:100CA8001D000323814690460293E3E600239A46FB
:100CB80004339846033B00250293DBE642460133A2
:100CC8001A432B0090465A1C0192424600240020E9
:100CD80001260A2A00DCEAE62CE70122D21A382A81
:100CE80000DDF4E61F2A00DC2AE11F214942CB1A65
:100CF8002100D9400B00202A05D0164A019D9446B0
:100D08006544AC402043421E904118430723190014
:100D18000024014003420CD00F230340042B00D1D0
:100D280040E1031D8342A441180064426107640244
:100D3800240BC20800230A43CCE6C046FF07000084
:100D480001FCFFFFFF030000FFFFFFFEFE0700009E
:100D58000DFCFFFF3E04000049464A460904090C01
:100D68000D00160C020C0004000C4543AC460500AF
:100D78007543A84615000F007543009202952A0096
:100D8800009D6F4365462D0CA94647444F44B8451E
:100D980005D91500802252029046454402953D0C23
:100DA800039565462D043F042D0CAC463D00654473
:100DB8000495250C2404240CAC4625007543A8464C
:100DC80065460F006943414489466743390C4944E5
:100DD8006E43884503D980225202904646440D0C42
:100DE800A846350045440595039D3F04A8463F0C99
:100DF8000904C91988444546039555462E04360CFE
:100E08002F0C35004543784381463800A8462D0C01
:100E1800AA46009A504372434A445244914503D922
:100E280080256D02A9464844150CA94645462D045F
:100E38002D0CA84665467D43120448449044A946B3
:100E48003200654662436E437C43170C3619BF195E
:100E5800BC4203D980246402A446E144029C039E58
:100E6800A446059D66448E428941AC4612043C0462
:100E7800120CA2186244494254184644A4464645F6
:100E8800A44182466442A046AA4292418C458941C7
:100E9800E244D044494252420A43A045A441824513
:100EA8008941644249420C4341463F0CD219121908
:100EB800CC0D049970020843411E884141464A44BA
:100EC800F60D52023043490214430843D20135D586
:100ED8000122430802401343E0071843640834E63C
:100EE800009BA2469B4681468024534624031C430C
:100EF80024034A462E4B240BECE500F0C7F81523D3
:100F08009C4684440200634620321C2B00DC84E6A5
:100F1800002399462300083883409A468EE600F05D
:100F2800B5F802000300153220331C2A00DC4EE617
:100F380002003400083A0020944052E6019304E687
:100F48001C4B21009C460300019DD3406544A940E9
:100F580019430300AB40581E834119430800D4408D
:100F68004B0709D00F230B40042B05D00B1D8B42D8
:100F78008041404224181800230200D4D6E60123F9
:100F880000240022A6E50F29AAD1802352461B037C
:100F98001A42A9D01C42A7D11C43009B02009B46C1
:100FA800034B97E50024C1E60024014B220091E59C
:100FB800FF0700001E0400000B00020070B5164D6C
:100FC8000C0382B04900002000920193240B490DC4
:100FD800DE0FA94204DD1148814203DD104BF018F1
:100FE80002B070BD8020400320430E4C641A1F2CB1
:100FF80008DD0D4B5B1AD84003005842002EEFD194
:101008001800EDE7094B009A9C46030061448B40A9
:10101800E2401343F1E7C046FE0300001D04000050
:10102800FFFFFF7F3304000013040000EDFBFFFF08
:1010380070B5002816D0C317C5185D40C40F280026
:1010480000F024F8104B1B1A5B055B0D0A2814DC12
:1010580002002E00153296400B22121AD5402D039D
:101068002D0B03E000240023002500261B052B433D
:10107800E40723433000190070BD0B3885402D0369
:1010880000262D0BF2E7C0461E0400001C21012398
:101098001B04984201D3000C10391B0A984201D353
:1010A800000A08391B09984201D30009043902A231
:1010B800105C40187047C046040302020101010198
:1010C800000000000000000010B584B00C220021D0
:1010D80001A805F003FA1A4C1A4B04222360802356
:1010E8002C21DB026261033A625463600021002311
:1010F800A276E26106326263A26320003532A36001
:10110800E360236123836362A3622363A154E364DE
:1011180000F04CFC00280CD10B4B2000019300235D
:1011280001A90293039300F0B7FD002804D104B08D
:1011380010BD00F0B1F9EFE700F0AEF9F7E7C046EF
:101148009C000020002401400200000470B5040047
:101158008EB01422002102A805F0C0F91C2200213B
:1011680007A805F0BBF9274B22689A4201D00EB0B8
:1011780070BD8023DB010793802307A81B060C930F
:1011880002F0C2FD002837D180211F4B49031A6C99
:10119800A0200A431A641A6C00260A400092009A9A
:1011A8000122596BC005114359635B6B02A91A40B0
:1011B8000192019B0222032304960292039301F0F9
:1011C800C5FB124D124B28002B6005236B607B3347
:1011D8002B6180336B618023DB00AB612023EB61E3
:1011E80080235B01AE60EE602B6201F09BF8002863
:1011F80005D12565AC62BAE700F04EF9C4E700F006
:101208004BF9F6E70024014000100240400000209E
:101218000800024001230E4A00B5916B83B01943C0
:101228009163926B00211340019300220920019BD6
:1012380000F0F8FF092001F01FF8002200210A2021
:1012480000F0F0FF0A2001F017F803B000BDC04617
:1012580000100240F0B589B01422002102A805F060
:101268003DF902220124C826A0252A4B2A4F596B92
:10127800B60011435963596BED050A400092009A74
:101288005A6B310022435A635B6B38002340019349
:101298000122019B01F0DEFC00222800202101F040
:1012A800D9FC02960026380002A9039404960594F6
:1012B80001F04CFB8823882228005B0302A90292D4
:1012C8000393049601F042FB20232800029302A90D
:1012D8001D3B05930394049601F038FB002340223C
:1012E800280002A902920393049601F02FFB002222
:1012F8000021062000F096FF062000F0BDFF002226
:101308000021072000F08EFF072000F0B5FF09B08C
:10131800F0BDC046001002400004005010B5194B43
:10132800194C01222360194B200063600023E260FE
:10133800A36023616361A361E361236201F0E0FDBF
:1013480000280CD10021200002F0D2F800280ED18C
:101358000021200002F0F2F8002810D110BD00F0A2
:101368009BF80021200002F0C3F80028F0D000F01C
:1013780093F80021200002F0E1F80028EED000F0F8
:101388008BF8EBE70058004000010020BC7D70108E
:1013980010B5040088B01422002102A805F09EF8B8
:1013A800124B22689A4201D008B010BD0123104C9C
:1013B800A020626B02A91A436263626BC0051340E6
:1013C8000093C022009B122352010292039306232A
:1013D800069301F0BBFA8022E36BD2031343E36365
:1013E800E36B13400193019BDEE7C04600580040C1
:1013F8000010024000B593B03422002105A805F082
:101408006DF810220021684605F068F880208000F9
:1014180002F0C2F8022305930C930D9306330F9341
:10142800C0238022DB0252001093802340210892BF
:1014380000229B0505A809920A910E92119302F0C9
:10144800DBF8002801D072B6FEE7072202230092DB
:10145800019300220023022168460292039302F0BE
:1014680077FB002801D072B6FEE713B000BDC04676
:1014780010B500F057FAFFF7BDFFFFF7EBFEFFF7D7
:10148800C9FEFFF721FEFFF749FF00F0C5F800F09D
:1014980005F904F00BFFFEE772B6FEE701220C4BDC
:1014A80000B5196CC02011431964196C83B00A4047
:1014B80080210092009ADA6B49050A43DA63DB6BF4
:1014C800C0000B400193019B00F064FA03B000BD1B
:1014D80000100240FEE7C046FEE7C0467047C0461F
:1014E8007047C04610B500F031FA04F06FFF10BD28
:1014F80010B5082001F0BCFB10BDC04610B5802017
:1015080001F0B6FB10BDC04610B5024801F0A6F8C0
:1015180010BDC0464000002010B5034801F09EF8F9
:10152800024801F09BF810BDFC010020A00100203A
:1015380070B5134C200003F0C1F9200003F0C8F87F
:1015480010222368D9690A4204D01A620D4B1A780E
:10155800002A07D00C4D802229002000520003F0F9
:1015680031FE70BD094A084D1268290052680848C2
:101578005242D2B21A701A78D2B204F0DBFFEAE70C
:10158800580200209008002090070020FC0100204D
:10159800900500207047C046084B026882B09A4206
:1015A80001D002B070478021054B09021A6C0A432A
:1015B8001A641B6C0B400193019BF2E7002000406A
:1015C8000010024010B5040088B01422002102A8BF
:1015D80004F084FF0E4B22689A4201D008B010BD77
:1015E80001230C4AA020516BC00519435163526B6B
:1015F80002A9134001931022019B02230292039334
:10160800022305930233069301F0A0F9E6E7C046EA
:10161800002000400010024010B588B01C220021B4
:10162800684604F05BFF1B4C1B4BFA222360142313
:101638006360002392002000A360E2602361A3613D
:1016480002F06AFE002818D1200002F095FE00285A
:101658001AD1AF2360229B0000920193002300223D
:10166800694620000293049302F0F6FE00280ED18A
:101678002000FFF7A7FF08B010BDFFF70DFF2000FF
:1016880002F07AFE0028E4D0FFF706FFE1E7FFF753
:1016980003FFEDE7540100200020004010B5214B66
:1016A800214C0C22236096239B01636000232000B9
:1016B800A360E36023616261A361E3612362636203
:1016C800A36203F0F5FC002811D10021200003F0EB
:1016D800E9FD002813D10021200003F00DFE0028A9
:1016E80015D1200003F0C2FD002817D110BDFFF767
:1016F800D3FE0021200003F0D5FD0028EBD0FFF732
:10170800CBFE0021200003F0F7FD0028E9D0FFF709
:10171800C3FE200003F0AAFD0028E7D0FFF7BCFEB7
:10172800E4E7C046003801405802002070B50400C4
:101738008EB01422002102A804F0D0FE1C22002141
:1017480007A804F0CBFE364B22689A4201D00EB0AF
:1017580070BD012307A8079302F0D6FA002856D1D6
:101768008021304BC9011A6C00260A431A641A6C8E
:101778002D480A400092009A0222596B114359637E
:101788005B6B02A91A400192019BC02202230292BC
:1017980003930023002206960492059301F0D6F8DD
:1017A800224D234B28002B6032236B604E332B6174
:1017B80080239B01AE60EE606E61AE61EE612B62CC
:1017C80000F0B0FD002828D180221A4BA550AC6249
:1017D800194D2B6033236B60233BAB600023EB6018
:1017E8006B61AB61EB61802328009B012A612B624E
:1017F80000F098FD00280DD1002200211B20E5678C
:10180800AC6200F00FFD1B2000F036FD9FE7FFF7EC
:1018180043FEA5E7FFF740FEEEE7FFF73DFED3E7FF
:10182800003801400010024000040050FC01002074
:101838001C00024030000240A00100200D4B02684D
:1018480010B504009A4200D010BD0B4A0B49136C26
:101858000B480B401364C02101F06AF98023E0585B
:1018680000F0D6FDE06F00F0D3FD1B2000F010FD66
:10187800EAE7C0460038014000100240FFBFFFFF02
:10188800000400500D488546FFF784FE0C480D49BA
:101898000D4A002302E0D458C4500433C4188C42C3
:1018A800F9D30A4A0A4C002301E013600432A24229
:1018B800FBD304F01BFEFFF7DBFDFEE700900020E2
:1018C8000000002024000020D0660008240000202A
:1018D80018090020FEE7000070B50F4B04001978C6
:1018E800002901D1012070BDFA208000FEF70CFC10
:1018F8000A4D01002868FEF707FC00F0D9FC002813
:10190800F0D1032CEED801380022210000F08AFC27
:10191800034B00201C60E6E70400002000000020C4
:10192800080000208023084A5B00116810B50B43AB
:1019380003201360FFF7D0FF041E02D0012420000B
:1019480010BDFFF7ABFDFAE700200240034A044B45
:1019580011681B785B1813607047C046EC020020C2
:1019680004000020014B18687047C046EC020020B4
:1019780070B50400FFF7F6FF0500631C02D0044BA6
:101988001B78E418FFF7EEFF401BA042FAD370BDA6
:1019980004000020034A044913680B400343136002
:1019A8007047C04600000140FFF9FFFFF0B5D6467A
:1019B8004F4646460023C0B582B0041E01932CD082
:1019C800856D002D00D1CCE0802325685B05AA68D1
:1019D8001A4215D1AA687B490A401343AB607A4B77
:1019E8007A491868FEF790FB013040000190019B8E
:1019F800002B05D0019B013B0193019B002BF9D1E2
:101A0800AB680020DB0000D49DE0AB685B070BD51A
:101A1800A36D1022A36D1343A365012002B0E0BC9F
:101A2800BA46B146A846F0BDA36DDB06F1D4A36D56
:101A3800674A216913400632FF321343A365AB6836
:101A4800DB075CD4276BA2687B1E9F41E368A67EF8
:101A58001A43237E3F039B031A43637EDB031A4327
:101A680073031A43002900DA9BE080239B039C46FA
:101A78002C23E35C5B0013433B436246202713435C
:101A8800E25D012A00D190E0626A002A05D0E026D2
:101A980076003240A66A324313433C27EA684D4E2B
:101AA800324013436668EB60E26CE75DB30F9B0757
:101AB8009A46BC461A43012F09D1676C236C3B43F5
:101AC8001A435346A76C3A431A4363461A432B6991
:101AD800414F3B40134380222B6173005B08D205C2
:101AE80093420CD080231B069E4208D03B4A3C4FB1
:101AF80013683B40F027BF033E403343136007267B
:101B080070276B69626BB34313436B616E69A36B98
:101B1800BE431B0133436B61002928D11023A96AF6
:101B28005B420B43AB62072369690B409A422FD093
:101B38001222A36D9343023A1343A365E36D0F3A50
:101B48001343E36569E71022A36D01201343A365DE
:101B5800E36D0F3A1343E365AB685B0700D463E7B3
:101B680056E7FFF7F3FA5423E565E5542CE780239D
:101B78009B039942D7D11C21AB6AE369013B9B00C7
:101B8800194010235B428B40216E0B43AB62CAE7BE
:101B980000230322E365A36D9343023A1343A3652D
:101BA8003CE74B005B089C4662E7002E03D180228D
:101BB8005202134368E7A66D3E43A665E66D3243BD
:101BC800E26561E7E8FFFF6F00000020400D0300B9
:101BD800FDFEFFFF0102DEFF02FCFF1F0827014098
:101BE800FFFFC3FF7047C0467047C04610B5806A04
:101BF800FFF7FAFF10BDC0467047C0464022806A12
:101C080010B5836D13438365C36D3C3A1343C365B5
:101C1800FFF7F2FF10BDC04650210300806A10B5DF
:101C2800826D11420DD18023826D9B001343C02227
:101C3800836503681201D96811420AD0FFF7D2FF01
:101C480010BD826DD20616D4026D1800526B9047F3
:101C5800F6E7827E002AF1D11A681207EED59A6853
:101C680052070BD52022836D13438365C36D1F3A3A
:101C78001343C365E2E7FFF7BFFFE1E70C215A68AA
:101C88008A435A60836D034A13400432FF32134378
:101C98008365D3E7FEFEFFFFF0B5DE4657464E46A6
:101CA800454600230400E0B585B003935433E25C55
:101CB8000069012A00D19AE00122E2542368033224
:101CC8009E6832420ED00120A36D1C321343A365D7
:101CD80054230022E25405B0F0BCBB46B246A946E4
:101CE800A046F0BD4E68904384460868022E5ED038
:101CF80047037D0B802700953F06BC4553D0276ED0
:101D0800BB461F27B8463740BA460F275546AF404F
:101D1800FD43BC4601955F466546AF43009DB94605
:101D2800002D66D14546820E15402A005546AA4028
:101D38004D461543A9464A46B6082266E269013669
:101D4800964208D856468200120FB2409D6A019EFC
:101D580035402A439A6205028A6829005E692A404A
:101D6800664D8E432A4032435A61002801DB002029
:101D7800AEE7E021624D634A2B684904194090425E
:101D88004CD0614A904240D0604A9042EFD18022C4
:101D9800D2031342EBD12B685D4803400B431A432F
:101DA80000202A6094E79A6A2A439A62D3E780223D
:101DB8001206944504D19A6A4103490B8A439A62F0
:101DC8000028D4DA4E4A4F491368884223D04E4936
:101DD80088424AD04D498842C9D1C0201168400480
:101DE80003404B4801400B430020136070E702207A
:101DF80071E7012505429ED1022707422DD05246A0
:101E080095404A462A43914695E780225204134258
:101E1800C1D000205CE7A0201168E0E7802212040E
:101E28001342A4D12B683A4803400B431A43394B59
:101E38002A6018683849FEF767F9013043001B1813
:101E48009B000393039B002B91D0039B013B0393BF
:101E5800039B002BF9D100203AE7024209D05246F1
:101E680097404A463A43914665E7C0201168000406
:101E7800B6E7020701D5032258E7C20601D50422B6
:101E880054E7820601D5052250E7420601D506220D
:101E98004CE7020601D5072248E7C20501D508220A
:101EA80044E7820501D5092240E7420501D50A2207
:101EB8003CE7020501D50B2238E7C20401D50C2204
:101EC80034E7820401D50D2230E7420401D50E2201
:101ED8002CE7020404D55A4665462A4391462AE768
:101EE800C20301D5102221E7820301D511221DE783
:101EF800420300D41FE7122218E7C04600FFFF077D
:101F080008270140001000B0004000B8002000B4CD
:101F1800FFFF3FFE00000020400D0300026870B57F
:101F2800936804005B0716D593689B0715D5FFF7E0
:101F380019FD236806009B685B070CD50425FFF78D
:101F480011FD2368801B022802D99A68154212D114
:101F58009B681D42F3D1002070BD93680B490B406C
:101F680010210B439360FFF7FDFC236806009B6874
:101F78005B07E3D4EFE71022A36D01201343A365A9
:101F8800E36D0F3A1343E365E6E7C046E8FFFF7FDA
:101F980000230122F0B583B0019303680400996817
:101FA8000A421FD19868284908421ED199682748D3
:101FB80001400A439A60264B1B681B020FD5254B2C
:101FC80025491868FEF7A0F801300190019B002B05
:101FD80005D0019B013B0193019B002BF9D1637E46
:101FE800012B0BD1002003B0F0BD1021A36D0120FF
:101FF8000B43A365E36D1343E365F4E7FFF7B2FC16
:10200800236806001A68D207ECD401250F4F9A6896
:10201800154203D19A683A402A439A60FFF7A2FC16
:102028002368801B022802D91A68154203D01A684F
:102038001542ECD0D6E71022A36D01201343A36507
:10204800E36D2B43E365CEE717000080E8FFFF7FD1
:102058000827014000000020400D0300F0B5C646E7
:1020680005680400AE6888461700022000B57607A8
:1020780014D45422A35C012B10D00123A354EA6882
:10208800134206D1AA68134231D10122EB681343E7
:10209800EB602000FFF77CFF002802D080BCB84628
:1020A800F0BDA26D154B256D1A4080235B001343CC
:1020B800A365134BE065EB62124B10222B63124BA6
:1020C80021686B631C230B603833E0544B6828008D
:1020D80013434B6042463B00403100F0FFF9226851
:1020E8000A4993680B4004210B439360D6E7AB6819
:1020F800064A13400343AB60C7E7C046FEF0FFFF44
:10210800211C0008F51B0008051C0008E8FFFF7FDC
:102118000222F8B50368040099680A4202D09B6855
:102128000020F8BD012198680142F9D00527986878
:102138000740012F08D01022A36D01201343A36587
:10214800E36D0B43E365ECE799681248012501400C
:102158000A439A6003221A60FFF704FC236806000A
:102168009B681F42DCD0FFF7FDFB2368801B022819
:1021780002D99A68154203D19B681D42F3D1CFE773
:102188001022A36D01201343A365E36D2B43E36580
:10219800C7E7C046E8FFFF7F542370B5C25C040060
:1021A800012A25D00122C254FFF7B8FE051E1AD114
:1021B8002523206DC35C022B1CD01021226820002F
:1021C80053688B435360FFF7A3FF051E06D1A36D29
:1021D800134A13400432FF321343A36501212268D6
:1021E800D3688B43D36054230022E254280070BD87
:1021F8000225FBE700F0BAF9051EDED040221021C7
:10220800A36D200013432268A36553688B43536072
:10221800FFF77EFF01212268D3688B43D360E2E792
:10222800FEFEFFFFFF22032310B514000340DB006E
:102238009C4089010A40E4439A4000280BDB0C4B80
:10224800C0219C4680088000604489004358234090
:102258001343435010BD0F23064903408C46083BE7
:102268009B089B006344D9690C401443DC61F1E787
:1022780000E100E000ED00E0002805DB1F2201235B
:1022880002409340014A13607047C04600E100E0F5
:1022980000280ADB1F2201230240934080220349C1
:1022A8008B50BFF34F8FBFF36F8F704700E100E093
:1022B8008022431E5204012093420ED2C021074AB5
:1022C80007485360036A09061B021B0A0B43036293
:1022D80000230020936007331360704710E000E08C
:1022E80000ED00E0F0B5846CC56C6560046D002CF1
:1022F80002D0446D856D65601C24056C084E254030
:102308001B3CAC4077683C43746004686360836836
:10231800102B02D0A160E260F0BDA260E160FBE793
:1023280000000240F0B5C646040000B5002860D0A1
:102338000568314B1421E818FDF7E6FE8300236495
:1023480002222523E2542B682C4AA66813402B60EE
:10235800E368216933430B4361692A680B43A16928
:102368000B43E1690B43216A0B4313432B60244B56
:1023780014219C4660448700FF20224B2840A36418
:10238800676408389846FDF7BFFE1F230122034003
:10239800100098408023E064DB019E421FD03F2359
:1023A800454661680B4001393B60686003291BD8CA
:1023B800154916485918013B9A40002389002165A0
:1023C8006065A2650B604260002325220121002080
:1023D800E363A154013AA35480BCB846F0BD00237E
:1023E80063603B6043465860002323656365A365CB
:1023F800EAE70120F0E7C046F8FFFDBF0F80FFFFC6
:1024080000820010800802403F820010400902400C
:10241800F8B5CE464746040080B500284FD003687B
:102428000126984642461B682648B3431360142188
:102438004044FDF769FE00274346810021641F6080
:102448001C230B40310099400B001F4A142155688A
:102458002B4353601D4BC5181D4BFF209946A364A1
:102468004346AD00184065640838FDF74DFE1F234C
:10247800320003409A401300E2644A462F605360DA
:1024880063685A1E032A11D90023252200202365D8
:102498006365A365E36223636363A363E363A35490
:1024A800013AA354C0BCB946B046F8BD09499640A4
:1024B8008C4663449B001F60074B5E60E4E7012085
:1024C800F0E7C046F8FFFDBF0000024000820010A0
:1024D800800802403F82001040090240F8B504001D
:1024E8002420255C012D35D0012525262554A55D00
:1024F800EFB2012D05D08023E3630023235401208C
:10250800F8BD2238A05500202568E0632868B84344
:1025180028602000FFF7E6FE236B002B1CD00E225C
:102528002B6813432B60626C1368DB0304D580238C
:1025380011685B000B431360236D002B04D08022CD
:10254800196852000A431A6001222B6800201343BD
:102558002B60D5E70220D3E704222B6893432B6036
:102568002B68063213432B60DDE7C04670B50028A0
:1025780032D02523C35C022B29D10E210268174CC7
:1025880013681C268B43416C13600B6823400B6057
:102598000123116899431160026C1149324093403C
:1025A8004D682B434B60C26C836C5A60036D002BE3
:1025B80005D01A6822401A60436D826D5A6025233F
:1025C8000122C2540022013BC254002070BD0423E2
:1025D8000022C3632033C2540120F7E7FFFEFFFF48
:1025E80000000240252370B5C35C022B03D00423EE
:1025F800C363012070BD0E2102681C261368154CA8
:102608008B4313600123116899431160416C0A6878
:1026180022400A60026C1049324093404D682B43B7
:102628004B60C26C836C5A60036D002B05D01A682E
:1026380022401A60436D826D5A6025230122C254DC
:102648000022013BC254836B002B00D09847002026
:10265800D0E7C046FFFEFFFF0000024070B51C2116
:1026680004242B4B06681A68036C35680B4021005C
:1026780099400A4210D02C420ED033689B0602D4EF
:102688003368A3433360224B5A6811435960036B84
:10269800002B00D0984770BD0224210099400A42BF
:1026A80017D02C4215D033689B0606D40A2233680B
:1026B800934333602523093AC254154B5A68114392
:1026C800596000222423C254C36A002BE3D09847E0
:1026D800E1E708210C009C402242DCD02942DAD0F4
:1026E800326806318A433260012215009D402B0072
:1026F80007494C6823434B602523C263C254002218
:10270800013BC254436B002BC5D09847C3E7C04672
:10271800000002402523C05CC0B27047C06B704700
:10272800054B00205A69002A05DA044A9A60044ACF
:102738009A605869C00F704700200240230167451E
:10274800AB89EFCDF8B504008026FFF70BF9174DDC
:102758000700760201E0631C15D12B693342FAD1D8
:102768002A69134B10001349184029611A4218D1DD
:1027780080250E4EED0201E0631C0BD133692B421C
:10278800FAD10020F8BDFFF7EDF8C01BA042E4D352
:102798000320F7E7FFF7E6F8C01BA042EED30320BB
:1027A800F0E7054B58600120ECE7C04600200240E6
:1027B800FA830000FB830000F0020020F0B5C64653
:1027C800244F14003A7880460D001E0000B5012AF7
:1027D80024D00123FA203B70002380007B60FFF7A0
:1027E800B1FF002804D000233B7080BCB846F0BD80
:1027F8004346194A012B13D1414653690B43536190
:102808002C60BFF36F8F6E60FA208000FFF79AFF8D
:102818004146114A53698B435361E4E70220E4E7D8
:1028280080235169DB020B435361EFF3108072B6CA
:10283800661CFF362D1B23682B510434A642FAD19F
:102848008022054952020B691342FCD180F310889B
:10285800DAE7C046F002002000200240FA2010B556
:102868008000FFF76FFF8022044B120659690A4364
:102878005A615869C043C00F10BDC04600200240CD
:10288800F0B54F464646D6462B4B050098461B7872
:102898008946C0B5012B41D042460123FA20137066
:1028A800002380005360FFF74DFF071E2DD104233E
:1028B8006B602B68042B33D001234A465B421360BC
:1028C800AC68EB68E3189C421AD21C4B1C4E9A4623
:1028D80005E0AB68EA6801349B18A34210D9514659
:1028E800FA207269E3000A401343164A8000134332
:1028F8007361FFF727FF0028EBD04B4607001C60E9
:1029080002210F4A53698B435361002342461370D7
:102918003800E0BCBA46B146A846F0BD0227F7E742
:10292800FA20074A084B516980000B435361FFF7AF
:1029380009FF0700E9E7C046F002002007E0FFFFB3
:10294800002002400200010004000100F0B5DE464C
:1029580057464E464546E0B50C688B46002383B083
:10296800002C68D001229A40944622409246624642
:1029780014425CD003215A465F00B94055680322CF
:10298800C9432A40561E0091012E5BD9032A00D064
:10299800ADE0BA400668009931400A430260C0229F
:1029A8009202154243D003270F265D491F408C46EB
:1029B800FF00BE409A0892006244116EB143A026FF
:1029C800F605B0420ED0574EB04200D1A0E0564EA8
:1029D800B04200D1A0E0554EB04200D194E00526A7
:1029E800BE4031438026116651464D4A7603C9439D
:1029F8001268354200D077E00A40494E326072686A
:102A08008026B60335426CD10A40454E7260842256
:102A1800B258AF0362D40A408427414EF251802253
:102A2800B258ED0356D40A4080213D4D6A50220029
:102A38000133DA4096D103B0F0BCBB46B246A94692
:102A4800A046F0BD81680E0000990E405946C9683D
:102A5800B1460E00BE40B0464E4641460E43866023
:102A680041680E0061468E432909B0460E000121D7
:102A78000E409E40B446464661460E434660C168D5
:102A88000E0000990E4059468968B0460E00BE40B7
:102A9800B446464661460E43C660022A00D078E72F
:102AA800D90889008C46844461460E6A072119407A
:102AB8008900884601960F214646B140019E8E4303
:102AC8005946019646460969B140019E0E43614642
:102AD8000E625EE7514611430A00A5E756463243A7
:102AE8009AE75646324390E75646324385E7C1682F
:102AF800009E3140884659468968B9408C4641460F
:102B080066463143C16044E70326BE40314369E766
:102B18000126BE40314365E70226BE40314361E7E6
:102B2800001802400004005000080050000C00503B
:102B3800F0B5DE4657464E464546E0B5002383B01D
:102B4800002965D001229146023293463A4A9446BA
:102B580044E03A4CA04262D0394CA04263D0394C90
:102B6800A04264D00524AC402500AE4214D1802494
:102B7800654666462D59BD43355104343559BD4324
:102B8800355144467568BD4375603568BD43356049
:102B9800019E356EA54335665E465D00AE4004680D
:102BA800350034430460DC08A4000419266A0727AA
:102BB800B0460F261F40BF00BE4037004646BE4302
:102BC80026628468AC438460446894434460C26865
:102BD800AA43C2600A000133DA4019D04A460F00FE
:102BE8009A4017401142F5D0134D9C08A846A400FE
:102BF8005D464444266E01940F241D40ED00AC4010
:102C0800A0462640A024E405A042A2D10025ACE7B6
:102C180003B0F0BCBB46B246A946A046F0BD4C4640
:102C2800AC402500A1E70224AC4025009DE75C46A6
:102C3800AC40250099E7C046001802400004005047
:102C480000080050000C005000690840431E9841DD
:102C5800C0B27047002A01D0816170478162FCE7E9
:102C6800426913000B401B0491430B438361704777
:102C78000B4B10B5DA680400104204D1084B1A69EE
:102C8800224207D110BDD86003F0E0F9044B1A695D
:102C98002242F7D020001C6103F0EEFAF2E7C046AA
:102CA80000180240F0B516001022C6461500036849
:102CB8000F009969040000B500200D400A4212D0A7
:102CC8002025DA6128009A691040154200D073E087
:102CD8007A1C45D120219A691142FCD02022DA6160
:102CE80004250543012080219A6949000A422CD015
:102CF8000120D9610543510504D508210D438021E0
:102D0800C900D961920504D502221543FF32FF326A
:102D1800DA619A69920701D500229A6201229969BB
:102D28000A4219D05A68254901200A405A60636C42
:102D380020222B4363644123E25400232232A3540C
:102D4800023AA35480BCB846F0BD5105D5D49205CB
:102D5800DAD40028F6D0DCE799690A439A61E1E7FA
:102D6800FEF700FE2368801BB84201D8002FA9D1C6
:102D780042225868A25C9969D2B2090403D580211D
:102D8800C90108420ED02022904641469A69114254
:102D980098D1FEF7E7FD2368801B1928F5D9202074
:102DA8009A699DE7202AEED05A6811435960FEF7C8
:102DB800D9FD23680600E6E700208FE700E800FE5B
:102DC800F8B504000D0016000227036809E0320078
:102DD80029002000FFF766FF00281FD16B1C05D1D2
:102DE80023689B691F42F2D00020F8BDFEF7BAFDA8
:102DF8002368801BA84201D8002DF2D102210800C7
:102E08009A6910401142ECD12022636C1343636429
:102E18004123E2540133E054023BE0540120E4E74B
:102E2800F8B54746CE4680B51F00089B0600994670
:102E38000D009046036809E04A4639003000FFF764
:102E480031FF002829D17B1C0CD133689C692C40A8
:102E5800641B63425C414445EED00020C0BCB946C7
:102E6800B046F8BDFEF77EFD4B46C01A3368B8423F
:102E780001D8002FEAD19A692A40521B51424A418F
:102E88004245E3D12022736C134373644123F25407
:102E980000232232B354023AB3540120DEE7C0467D
:102EA800F8B5036806009B690C00170020259B06EF
:102EB80010D518E0FEF756FD3368C01BA04201D8B4
:102EC800002C04D129009A69114015420DD09B6944
:102ED8001D4208D13A0021003000FFF7E3FE002828
:102EE800E8D00120F8BD0020FCE7736C2B43736425
:102EF8004123F5540133F154023BF154F1E7C04644
:102F080010B5041E52D04123C35CDAB2002B48D05E
:102F1800412324220121E2542368A0681A688A43C5
:102F28001A60234962680A401A619A6821490A406E
:102F38009A60E268012A0BD0842109020143996052
:102F4800022A09D18022596812010A435A6007E00F
:102F58008022120202439A605A6817490A405A604E
:102F68005968164A00200A435A60DA6811490A402B
:102F7800DA60616922690A43A16909020A43DA60D1
:102F8800216AE2690A4301211A601A680A431A6031
:102F9800002341221F316364A15401322363A354E7
:102FA80010BD4033C254FEF7F3F9B1E70120F7E74B
:102FB800FFFFFFF0FF7FFFFFFFF7FFFF008000022A
:102FC800F0B557464E46DE464546E0B583B01F008D
:102FD8000CAB160004CB04001B880D009B46412354
:102FE8009946C35C9246202B23D1002A1DD05B460C
:102FF800002B1AD04022835C012B1AD00123835462
:10300800FEF7B0FC802180460090192301222000A1
:103018000902FFF705FF00280DD0012003B0F0BC1E
:10302800BB46B246A946A046F0BD80239B00636418
:10303800F3E70220F2E721234A46A3544022213332
:10304800E254534663625B462168606463854A685C
:1030580060635448FBB20240AD051B041343AD0D39
:10306800514A2B4313434B60424620000E99FFF709
:10307800A7FE002857D12368012F63D1F6B29E62BC
:10308800434600220093802120000E9BFFF7C8FED4
:10309800002848D1638D2268FF2B48D8638D4348A8
:1030A8009BB251682385DBB21B0401402B430B43C1
:1030B800802189040B434646536002E0638D002B50
:1030C8005AD0320020000E99FFF77AFE0028A4D1CA
:1030D800636A22681978013391626362638D013BE8
:1030E8009BB26385238D628D013B9BB22385002AA9
:1030F800E4D0002BE2D10022802120000E9B009614
:10310800FFF78EFE002800D087E7638D2268FF2B2B
:1031180023D9FF232549238553680B4024492B4392
:103128000B435360CAE740230022E25475E7FF23AC
:103138001E492385536846460B401D492B430B43C4
:103148005360BEE7320A9A62200042460E99FFF7A2
:1031580037FE0028E7D1236890E7638D13489BB2B8
:1031680051682385DBB21B0401402B430B438021AC
:1031780089040B435360A1E7320020000E99FFF742
:103188008FFE002800D048E720212368094DD96127
:103198005A682A405A604123E1540133E054023B03
:1031A800E0543BE7009800FC00200001009C00FC74
:1031B8000000FF0100E800FEF0B557464E46DE4627
:1031C8004546E0B583B01F000CAB160004CB0400E5
:1031D8001B880D009B4641239946C35C9246202BD1
:1031E80023D1002A1DD05B46002B1AD04022835CD5
:1031F800012B1AD001238354FEF7B4FB80218046AB
:1032080000901923012220000902FFF709FE002877
:103218000DD0012003B0F0BCBB46B246A946A0467B
:10322800F0BD80239B006364F3E70220F2E72223CA
:103238004A46A35440222033E254534663625B4615
:103248002168606463854A6860635648FBB202403F
:103258001B0413438022AD05AD0D92012B4313438C
:103268004B60424620000E99FFF7AAFD002859D16D
:103278002368012F65D1F6B29E624346002200936F
:10328800402120000E9BFFF7CBFD00284AD1638D1B
:103298002268FF2B4AD8638D42489BB25168238528
:1032A800DBB21B0401402B430B433F4946460B430B
:1032B800536002E0638D002B5DD0002204212000C2
:1032C8000E9B0096FFF7ACFD0028A2D123685A6A2E
:1032D800636A1A70628D636A013A013392B263625B
:1032E800238D6285013B628D9BB22385002AE1D044
:1032F800002BDFD10022802120000E9B0096FFF7D3
:103308008FFD002800D084E7638D2268FF2B23D926
:10331800FF232649238553680B4025492B430B433C
:103328005360C7E740230022E25472E7FF231D4998
:103338002385536846460B401E492B430B43536075
:10334800BBE7320A9A62200042460E99FFF738FD21
:103358000028E7D123688EE7638D14489BB2516833
:103368002385DBB21B0401402B430B4380218904D6
:103378000B4353609EE7320020000E99FFF790FD43
:10338800002800D045E7202123680B4DD9615A68F1
:103398002A405A604123E1540133E054023BE0548F
:1033A80038E7C046009800FC00240002009C00FC9E
:1033B8000000FF010024FF0100E800FEF0B55746B9
:1033C8004546DE464E461C00002392464122E0B5A3
:1033D80085B00393835C0500202B5FD103688020B0
:1033E8009E69000237000740064257D140202E5CF4
:1033F800012E53D0012689052E541C38A8548A0D55
:1034080091464946384A6F6411438B46E9685A46E3
:10341800012902D14946354A0A435A60FEF7A2FA01
:103428002023296880468A6988691340102202404F
:10343800134312D120271026631C08D0FEF792FAF6
:103448004346C01AA04231D8002C2FD029688B6976
:103458008A693B4032401343EED010268B691E42E6
:103468002FD0434600220093202123002800FFF795
:10347800D7FC002810D120212B68DE61D961039A7E
:1034880001320392039A5245C0D34123E9546B6C2D
:103498000B436B644023E854012000E0022005B090
:1034A800F0BCBB46B246A946A046F0BD2022412347
:1034B800EA546B6C012013436B6400224023EA54E6
:1034C800EDE7434600220093202123002800FFF760
:1034D800A7FC0028E0D120232A68D3614122AB54FD
:1034E8002033E854DBE7C046002800020020000231
:1034F800F0B54124035D8C46DDB2202B1AD140265D
:10350800835D012B16D024230127035503680A493C
:103518001A68BA431A601A680A401A60624619683B
:10352800114319601A683A431A60002305558355F8
:103538000020F0BD0220FCE7FFEFFFFFF0B5CE460C
:103548004746412480B5035DDDB2202B1FD14026BC
:10355800835D012B1BD02423012703550268B9463C
:1035680013680902BB431360136898464746094B22
:103578001F4039431160494613680B431360002309
:10358800055583550020C0BCB946B046F0BD0220A1
:10359800F9E7C046FFF0FFFF70B5134C134A2368E4
:1035A800002513400343236080239B00984201D0E9
:1035B800280070BD0E4B0F491B685800C01840000A
:1035C800FCF7A2FD80226369D2000130134202D1C8
:1035D800EEE7002805D0636901381342F9D10025C8
:1035E800E6E70325E4E7C04600700040FFF9FFFF67
:1035F8000000002040420F00F0B5CE46474680B597
:10360800040083B0002827D00368DA0711D53822D0
:10361800C0498868C9680240102A00D1CCE0082A4D
:1036280000D0CDE0BB4A1268920302D56268002A36
:1036380012D09A0732D53823B64A91680B40D16820
:10364800102B00D10BE1002B00D00DE113685B05B6
:1036580008D5E368002B05D1012003B0C0BCB946EA
:10366800B046F0BD51686369AB481B0201400B438B
:103678005360A84AA94913680B4021690B4313609A
:103688001368A74A9B045B0FDA40A6490A60A64B59
:103698001868FEF721F90028DED123681A076DD4CF
:1036A8005B0745D538239B4A91680B40202B00D1F6
:1036B800CCE080230020D16B5B058146194208D1FC
:1036C800D16B1943D163D26B13400193019B012342
:1036D80099468027954E7F0033683B4200D1FFE032
:1036E800A368012B00D1E5E0052B00D1C8E1012139
:1036F800884EF26D8A43F265F26D03318A43F265B2
:10370800002B00D0DAE0FEF72DF9022307009846D7
:10371800874D05E0FEF726F9C01BA84200D9EEE068
:103728004246F36D1A42F5D14B46012B00D163E1B5
:10373800E369002B20D03822764DA9680A40102A68
:1037480000D11DE1022B00D15CE12B68794A80266B
:1037580013402B60FEF706F9B604040005E0FEF7F7
:1037680001F9001B022800D9C9E02B683342F6D1C1
:10377800EB68714A1340EB6000206EE73822654D14
:10378800A9680A40182A43D0A369002B00D1B8E0E1
:1037980001222B6E022713432B66FEF7E3F806007F
:1037A80005E0FEF7DFF8801B022800D9A7E02B6EA2
:1037B8001F42F6D0236873E7C943890700D131E770
:1037C80080226368520293422BD0A021C9028B4207
:1037D80000D1FCE04F4D59492A680A402A602A68FE
:1037E80057490A402A60002B1FD1FEF7BBF88027F3
:1037F8000600BF0204E0FEF7B5F8801B64287ED8F7
:103808002B683B42F7D123689A0700D446E712E7B2
:103818002A6E920700D443E7A269002A00D03FE746
:103828001AE73C4A11680B431360FEF79BF88026A1
:103838000500384FB60204E0FEF794F8401B6428F0
:103848005DD83B683342F7D02368DDE7D36D9B072B
:1038580000D46DE7A368002B00D069E7FCE60D3BB8
:103868000B40022B00D1BCE0E3682A4D002B73D03B
:103878002B682A4A802713402269FF0013432B60D4
:1038880080232A685B0013432B60FEF76BF8060061
:1038980004E0FEF767F8801B022830D82B683B420B
:1038A800F7D06A6863691C491B020A4013436B60BE
:1038B8002368F3E61749CA6D1343CB65FEF752F840
:1038C800144B060098460227194D04E0FEF74AF803
:1038D800801BA84213D84346DB6D1F42F6D023E76E
:1038E80033683B433360FEF73DF8050033683B42DD
:1038F80000D0F5E6FEF736F8401B0228F6D903207B
:10390800ABE601222B6E022793432B66FEF72AF8BB
:1039180006001CE000100240FF80FFFFFFC7FFFF0A
:103928000024F4000000002008000020007000407F
:1039380088130000FFFFFFFEFCFFFEEFFFFFFEFF06
:10394800FFFFFBFFFEF70EF8801B0228D7D82B6E6F
:103958001F42F7D12368A3E62B68504A80271340FB
:103968002B60FDF7FFFFFF00060004E0FDF7FAFFFC
:10397800801B0228C3D82B683B42F7D123688DE609
:10398800012B00D168E60322E868216A02408A42D6
:1039980000D061E67022616A02408A4200D05BE68C
:1039A800FE21A26AC90101401202914200D053E6E9
:1039B800F822E16A920302408A4200D04CE6236B67
:1039C800400F4007C01A431E9841C0B245E6802107
:1039D800334BC90218680143196019680A431A6011
:1039E80023E713685B0555D4516863692D481B02AA
:1039F80001400B4353604AE6294A2B49D36B0B40DD
:103A0800D36395E62B68294A802713402B60FDF77E
:103A1800A9FFBF04060005E0FDF7A4FF801B0228EC
:103A280000D96CE72B683B42F6D1616A236AEA68E1
:103A38000B431F491A4E0A401343E26A1343226B91
:103A48001343A26A12021343EB6080232A685B04C3
:103A580013432B608023EA685B051343EB60FDF793
:103A680081FF80250400AD0405E0FDF77BFF001B06
:103A7800022800D943E733682B42F6D00020ECE552
:103A88000421074BDA6D0A43DA65DA6D03390A4314
:103A9800DA6513E7E368002BA6D1DDE5FFFEFFFF3B
:103AA80000100240FF80FFFFFFFFFFEFFFFFFFFE58
:103AB8008C80C11F3823224A10B591680B4205D16A
:103AC800136820489B045B0FD84010BD91681940CB
:103AD800082914D091681940102912D0916819400A
:103AE800202924D0906818401838431E9841164B56
:103AF80040421840FA23DB019C466044E5E713483E
:103B0800E3E7D368D168DB43D4684906490F640406
:103B18000131640E9B070DD00A48FCF7F5FA6043A3
:103B2800074BD968490F0131FCF7EEFACDE7802041
:103B38000002CAE70548FCF7E7FA6043F0E7C04629
:103B4800001002400024F4000083FFFF00127A00F6
:103B5800F8B5CE46474605000C0080B5002826D0AB
:103B68000722574E336813408B425ED32B689A075F
:103B78000ED55A0705D5E0225249D201886802437A
:103B88008A60504950488A680240A86802438A609F
:103B9800DB072BD56B684B4A012B00D17CE0022B4D
:103BA80007D0002B00D07DE01268520504D4012014
:103BB80037E012689201FAD50721424EB2688A436B
:103BC8001343B360FDF7CEFE382398463F4B0700FA
:103BD800994604E0FDF7C6FEC01B48453BD843465E
:103BE800B2681A406B68DB009A42F3D10722344E60
:103BF80033681340A34238D82B685B072DD4FFF7EE
:103C080059FF304B324A9B6832491B051B0F9B00FA
:103C18009B581F221340D8402F4B08601868FDF7A7
:103C28005BFEC0BCB946B046F8BD336893430B434E
:103C38003360FDF797FE07239846244B0700994603
:103C4800424633681340A34200D18FE7FDF78AFE4E
:103C5800C01B4845F4D90320E3E71A4A1F49936873
:103C68000B40E9680B439360C9E7336893432343E8
:103C78003360FDF777FE07239846144B07009946F3
:103C8800424633681340A342B6D0FDF76BFEC01B13
:103C98004845F5D90320C4E71268920300D58BE79D
:103CA8000120BEE7032B05D0D26D920700D583E72C
:103CB8000120B6E7126E920700D57DE70120B0E734
:103CC8000020024000100240FFF0FFFF88130000B0
:103CD800C86500080000002008000020FF8FFFFFD3
:103CE800064B07499B68074A5B045B0F9B005B58C0
:103CF8001F2110680B40D8407047C0460010024092
:103D0800A865000800000020F0B5D6464F46464694
:103D1800C0B50368040082B000209A0351D5802200
:103D2800564B5205D96B8246114200D184E0802758
:103D3800534D7F002B683B432B60FDF713FE0600B5
:103D480005E0FDF70FFE801B022800D97EE02B68F6
:103D58003B42F6D0494DC023EA6D9B001000A16993
:103D680018401A4222D0884220D08020EB6DEE6D98
:103D780040023043E865E86D424A434E1A403040FD
:103D8800E865EA65DB0711D5FDF7ECFD02239846E7
:103D98003E4B0600994604E0FDF7E4FD801B4845CC
:103DA80054D84246EB6D1A42F6D0A169334A3548D9
:103DB800D36D03400B43D365524600202368012A84
:103DC80049D0DA0706D503252C494A6DAA43656808
:103DD8002A434A659A0706D50C2528494A6DAA43FD
:103DE800A5682A434A659A0606D52449284D4A6D8E
:103DF8002A40E5682A434A655A040AD51F49656975
:103E08004A6D920092082A434A658022D20595425B
:103E180027D01B050AD5194A2169536D1D4C23402B
:103E28000B4353658023DB01994220D002B0E0BCEC
:103E3800BA46B146A846F0BDD96B1143D963DB6BCE
:103E480013400193019B01239A4670E752460320D1
:103E58002368012AB5D109490F4DCA6B2A40CA63A4
:103E6800AFE78022CD6852022A43CA60D1E7802397
:103E7800D1685B020B43D360D8E7C046001002400C
:103E880000700040FFFCFFFFFFFFFEFF88130000EB
:103E9800FFCFFFFFFF3FFFFFFFFFFFEF70B50124DC
:103EA800036A026A144DA2430262426884692C4084
:103EB8000D682C430225AB438D682B430F4DA84258
:103EC80008D00F4DA84205D00E4DA84202D00E4D85
:103ED800A8420BD10825AB43CD688E692B43042536
:103EE800AB430A4D15404A6932432A4342604A6847
:103EF80084614263036270BD8CFFFEFF002C0140A9
:103F0800004001400044014000480140FFFCFFFF21
:103F180070B5184A046A036A134003624268164B74
:103F2800C5691D400B681D43144B1C408B681B0260
:103F38002343134CA04215D0124CA04205D0124C7A
:103F4800A04202D0114CA04206D1114C4E69144037
:103F58008A6932431201224342604A68C561C263DA
:103F6800036270BD0B4C1C40CB681B0223430A4CF8
:103F78002340EAE7FFFEFFFF8CFFFEFFFFFDFFFF88
:103F8800002C01400040014000440140004801402D
:103F9800FFCFFFFFFFF7FFFFFFFBFFFF30B5144A1E
:103FA800046A036A134D134003624368C2692A40D6
:103FB8000D682D021543104A14408A6812032243E3
:103FC8000E4CA04208D00E4CA04205D00D4CA04289
:103FD80002D00D4CA04204D10C4C1C404B699B01F3
:103FE800234343604B68C5610364026230BDC04629
:103FF800FFEFFFFFFF8CFFFEFFDFFFFF002C0140FC
:10400800004001400044014000480140FFBFFFFF5D
:1040180030B5134A046A036A124D134003624368B9
:10402800426D2A400D6815430F4A14408A681204ED
:1040380022430E4CA04208D00D4CA04205D00D4C96
:10404800A04202D00C4CA04204D1054C1C404B6944
:104058001B02234343604B6845658365026230BD9C
:10406800FFFFFEFF8FFFFEFFFFFFFDFF002C01405B
:1040780000400140004401400048014030B5144A66
:10408800046A036A134D134003624368426D2A4071
:104098000D682D021543104A14408A681205224300
:1040A8000E4CA04208D00E4CA04205D00D4CA042A8
:1040B80002D00D4CA04204D10C4C1C404B699B0211
:1040C800234343604B684565C365026230BDC04603
:1040D800FFFFEFFFFF8FFFFEFFFFDFFF002C014018
:1040E800004001400044014000480140FFFFFBFF41
:1040F8003D2110B5425C0300D4B20120012A12D13F
:1041080001325A541B68DA682243DA600D4A934236
:104118000AD00D4A934207D00C4A934204D01A6839
:1041280022431A60002010BD9A6809490A40062AED
:10413800F8D007398A42F5D001211A6800200A43CD
:104148001A60F0E7002C01400004004000400140E4
:104158000700010010B5102903D8394A8B00D3583D
:104168009F464323C25C012A01D10222C254012086
:1041780010BD3E23C25C012AF9D10224C45403684D
:10418800DA682243DA601F2211401E3A8A40196A0F
:1041980091431962196A0A431A622A4A93423AD029
:1041A800294A934237D0294A934243D0284A934216
:1041B80040D0284A934233D001211A680A431A6032
:1041C8000020D5E73F23C25C012AD0D10222C25485
:1041D80003680420DA680243DA60D4E74023C25C4B
:1041E800012AC4D10222C25403680820DA680243B3
:1041F800DA60C8E74123C25C012AB8D10222C2545E
:1042080003681020DA680243DA60BCE74223C25C24
:10421800012AAAD0ABE78022596C12020A435A64D9
:104228009A680D490A40062ACAD007398A42C3D17A
:1042380000209DE78022596C12020A435A64BBE7AA
:1042480008660008002C014000400140004401407D
:104258000048014000040040070001007047C046C4
:1042680010B5FFF777FF10BD70B5244E03680A68D4
:104278008C684D69B04230D0214EB04216D0214EE4
:10428800B04217D0204EB0422BD0204EB04228D09A
:104298001F4EB04212D11F4E3340CE6833438026A2
:1042A800B3431D430560C462826224E07026B343B1
:1042B8004E683343174EC96833400B4380218B4304
:1042C8002B430360C4628262012343610269134283
:1042D80002D002699A43026170BD7026B3434E68EA
:1042E80033430C4E3340CE6833438026B3432B43CD
:1042F8000360C46282620B690363E5E7002C014036
:1043080000040040002000400040014000440140FB
:1043180000480140FFFCFFFF70B5041E2AD03D2372
:10432800C35CDAB2002B20D002233D25210063555F
:1043380001C9FFF799FF012348220020A3540A3A34
:10434800A3540132A3540132A3540132A3540132BD
:10435800A3540132A3540132A3540132A3540132AD
:10436800A3540132A354635570BD3C33C254FDF7C6
:1043780013F9D9E70120F7E770B5041E2AD03D23C9
:10438800C35CDAB2002B20D002233D2521006355FF
:1043980001C9FFF769FF012348220020A3540A3A04
:1043A800A3540132A3540132A3540132A35401325D
:1043B800A3540132A3540132A3540132A35401324D
:1043C800A3540132A354635570BD3C33C254FFF764
:1043D80045FFD9E70120F7E7102270B5046A036AA0
:1043E800174D93430362436882692A400D682D0282
:1043F8001543202294438A6812012243114CA0429B
:1044080015D0114CA04205D0104CA04202D0104C3F
:10441800A04206D10F4C4E691C408B6933439B0068
:10442800234343604B6885618363026270BD8024C7
:10443800A2431600CA68403C12013243A243E9E78E
:10444800FF8CFFFE002C0140004001400044014069
:1044580000480140FFF3FFFF3C2370B50D00C15C2D
:104468000400012900D184E00121C154142A03D891
:10447800414B92009B589F4601203C230022E25466
:1044880070BD066829003000FFF7F8FD8023726DC3
:104498001B0113437365736D384A0020134073651D
:1044A8002B69726D1B0213437365E6E706682900E2
:1044B8003000FFF7F3FC0822B36900201343B3610F
:1044C800B369043A9343B361B3692A691343B36187
:1044D800D3E7066829003000FFF77EFF8023B26922
:1044E8001B011343B361B369244A00201340B3612D
:1044F8002B69B2691B021343B361BEE70668290042
:104508003000FFF705FD0822F36900201343F3612B
:10451800F369043A9343F361F3692A691343F36136
:10452800ABE7066829003000FFF738FD8023F26901
:104538001B011343F361F369104A00201340F36130
:104548002B69F2691B021343F36196E70668290099
:104558003000FFF75DFD0822736D0020134373657B
:10456800736D043A93437365736D2A6913437365D6
:1045780083E7022084E7C0464C660008FFFBFFFF84
:1045880030B5EFF31084012282F310880168134DCF
:104598000B682B400B6084F31088EFF3108182F3D3
:1045A800108802680E4C93682340936081F310884A
:1045B800C36E012B0AD1EFF3108183F31088102406
:1045C80002681368A343136081F310888C232022A8
:1045D800C2500023C366436730BDC046DFFEFFFFFD
:1045E800FEFFFFEF70B5041E18D088262423012192
:1045F8000025835103681A688A431A601D605D604C
:104608009D60FDF71BF990230020E550043BA55160
:10461800E550083BE5662567E55470BD0120FCE7D9
:1046280013008822F0B5C6468258040000B5202A37
:104638002CD1002928D0002B26D080228068520156
:10464800904238D054222165A3520232A35232320A
:104658009046902640460027673AA7512250E06FBF
:104668002268002817D0174D8763C562164D283277
:104678000563164D4563FDF731FF00280AD0102366
:104688004246A3511033A350012000E0022080BC11
:10469800B846F0BD226840231362EFF310813F3B18
:1046A80083F310888020226893680343936081F322
:1046B80010880020EBE72269002AC3D1CA07C1D5B8
:1046C8000120E4E7BD470008114800082948000810
:1046D800882370B504008022C0580433E558236845
:1046E80099680A4201D021281ED09A6840231342B3
:1046F80001D1002070BD222DFBD1EFF310800122E3
:1047080082F3108821688A689A438A6080F3108847
:1047180080256059002803D0FDF728FF00283FD1E5
:104728002000FFF72DFFE4E7EFF31080012383F368
:10473800108821688B6893438B6080F31088E06F42
:10474800002803D0FDF712FF00281FD1EFF31080D7
:10475800012282F31088C02621680B68B3430B60DE
:1047680080F31088EFF3108182F3108822680F48D5
:1047780093680340936081F3108888232022E250D5
:1047880023689A6840231342B3D0B4E7E06FFDF77B
:10479800C5FF2028DAD1902310220320E250A9E790
:1047A8006059FDF7BBFF2028BAD1F4E7FFFF7FFF70
:1047B8007047C0462022030011001B6810B51B6813
:1047C800806A19401A4219D15623C152EFF3108C4E
:1047D8001F3A82F31088802401688B68A3438B609A
:1047E8008CF31088EFF3108182F310880268402060
:1047F80013680343136081F3108810BDFFF7D8FFD7
:10480800FBE7C0467047C04610B5806AFFF7FAFF5D
:1048180010BDC0467047C0467047C0467047C04686
:10482800F8B588218C23846A6558E05823689A680B
:10483800120601D5212D14D09B685B0601D52228CC
:1048480008D090221021A35820000B43A350FFF753
:10485800E5FFF8BD5E2300222000E252FFF790FE3C
:10486800EFE756230022E252EFF31086013282F37B
:104878001088C02725682B68BB432B6086F31088F7
:10488800EFF3108582F310882268054E9368334051
:10489800936085F31088202363502368CCE7C046D3
:1048A800FFFF7FFF00235E2210B5806A8352083A1B
:1048B8008352FFF7B3FF10BD7047C046F8B54546B1
:1048C800DE4657464E460268E0B5D369B74D040048
:1048D800116890682B4238D120251D4206D08026C9
:1048E80076050D400640354300D0EBE0E56E012D1E
:1048F80000D1AEE080256D032B421FD180221A42E1
:1049080006D080252D040A402840024300D0E0E06C
:1049180040221A4202D00A4200D0E9E01A0202D527
:104928004A0000D5F8E0DB0102D5002900DAF7E0FB
:10493800F0BCBB46B246A946A046F8BD4602DDD546
:104948002000156200F08CFCF2E7994E994D064064
:104958000D403543CAD001251D4208D0CF0506D5E4
:104968009027BC461562E7593D436746E551042543
:104978002F001F40BC460227A9461F4200D199E0DC
:10498800C50716D5902517626759A8464D463D4379
:104998004746E5516546002D0BD0042515628C3538
:1049A800A9466559A846022547462F433D004F466C
:1049B800E55108271F4208D020250D40354304D073
:1049C80090261762A5593D43A55180252D012B42FC
:1049D80007D04E0105D5902620271562A5593D43DD
:1049E800A55190256559002DA2D020251D4205D03E
:1049F80080235B050D4003401D436ED19026402760
:104A08002823A15995680B403D4020001D4300D143
:104A18008AE0FFF7B5FD23689B681F4264D0EFF377
:104A28001081012383F3108822689368BB43936045
:104A380081F3108880256059002855D05E4B836328
:104A4800FDF7D0FD002800D172E76059836B9847C5
:104A58006EE710261E4200D14CE70E4200D149E70E
:104A680040231800166292681040134260D08022DA
:104A78009446A2581068426892B2002A00D157E7BB
:104A88005C218B46615A914200D851E75E27E25378
:104A98002022170000680740B846024200D191E082
:104AA800022323675C33E35A2000C91A89B2FFF74F
:104AB80003FF3DE76546002D00D17AE7C50700D41E
:104AC80077E76AE7636F002B00D131E7200098474A
:104AD8002EE7A36F002BF9D12AE7636F002B8DD047
:104AE80020009847226889E72000FFF797FE1FE714
:104AF800EFF31080012383F3108821680B68934338
:104B08000B6080F310888823203AE25000232000AD
:104B1800A367FFF74DFE0BE7200000F0A5FB07E7B2
:104B2800200000F09FFB03E7FFF778FEA551FFE6A2
:104B38005C235E22E15AA35AA25A9BB2002A00D1F2
:104B4800F6E6C91A89B2002900D1F1E6EFF3108917
:104B580085F310882268136898464746174B1F400C
:104B6800176089F31088EFF3108985F3108822689D
:104B7800936898464746124B1F40976089F3108800
:104B88008C232022E250E0666067EFF3108085F303
:104B9800108822681368B343136080F310880223D7
:104BA80020002367FFF788FEC2E6C0460F08000012
:104BB8000100001020010004AD480008DFFEFFFFDF
:104BC800FEFFFFEFEFF3108985F310882068174F79
:104BD80001683940016089F31088EFF3108985F383
:104BE800108820688168A943816089F31088EFF3F1
:104BF800108985F31088206881689943816089F35A
:104C080010884C33E2504346E366EFF3108185F396
:104C1800108822681368B343136081F310886346D1
:104C2800E058FDF7A3FC5B46E15A39E7FFFEFFFFBA
:104C38000123806A10B50367C36E012B02D0FFF70A
:104C4800EBFD10BD5B33C15A4908FFF735FEF8E7A5
:104C580003001B6870B51A6820231900806A114088
:104C6800134227D15E228152EFF310855D3A82F319
:104C7800108804681C4E21683140216085F3108833
:104C8800EFF3108582F310880468A1689143A1604E
:104C980085F31088EFF3108482F3108840250168AB
:104CA8008A68AA438A6084F310888C228350C36E72
:104CB800012B0CD000230367C36E012B02D0FFF732
:104CC800A9FD70BD5B33C15AFFF7F6FDF9E7EFF3B5
:104CD800108183F31088102402681368A3431360BB
:104CE80081F31088E6E7C046FFFEFFFF70B50400B9
:104CF8002569A26823682A4365691968C0692A4337
:104D08004C4D024329400A431A605A684A49256AA9
:104D18000A40E1680A435A60A26999682A43474DE4
:104D280029400F250A439A60DA6A616AAA430A434E
:104D3800DA62434A934224D0424A93420CD0424A10
:104D4800934228D0414A934225D00120404BA36684
:104D580000236367A36770BD3E4B5A6D0C23134055
:104D6800082B3DD021D8002B15D0042BEDD1802362
:104D78001B0298423AD0FEF79DFE002813D0616AC4
:104D88001AE0344B5A6D03231340022B28D0032B0F
:104D98000DD0012BEBD080231B02984245D0FEF7A3
:104DA8009FFF0028EBD10020D0E70C2BCDD180232A
:104DB8001B0298421FD01800274B4900C95AFBF71D
:104DC800A3F965686B08C0182900FBF79DF9020074
:104DD800224B103A9A42B8D82368D8600020B5E729
:104DE80080231B02984223D01D48E5E7FEF762FEA8
:104DF8000028D8D0616A184B4900C95AFBF784F9D2
:104E0800656840006B08C0182900FBF77DF90200AF
:104E1800124B103A9A4298D8124B22680340000766
:104E2800400F0343D360002090E7FEF759FFDFE708
:104E38000B48E0E7F369FFCFFFCFFFFFFFF4FF1157
:104E4800003801400044004000480040004C004049
:104E58000100010000100240A0660008EFFF0000FA
:104E68000024F400F0FF0000836A30B51A0706D565
:104E78000168284C4A682240846B22434A60DA075A
:104E880006D50168244C4A682240C46A22434A6015
:104E98009A0706D50168214C4A682240046B2243D0
:104EA8004A605A0706D501681D4C4A682240446B7F
:104EB80022434A60DA0606D501681A4C8A682240FD
:104EC800C46B22438A609A0606D50168164C8A6824
:104ED8002240046C22438A605A060AD50168134DA1
:104EE8004A68446C2A4022434A6080225203944212
:104EF80009D01B0606D502680D4953680B40C16CE2
:104F08000B43536030BD4A680A4C2240846C2243EC
:104F18004A60EEE7FF7FFFFFFFFFFDFFFFFFFEFF99
:104F2800FFFFFBFFFFEFFFFFFFDFFFFFFFFFEFFFCD
:104F3800FFFFF7FFFFFF9FFFF0B54F464646D646F7
:104F4800C0B5994680460D001600089F036801E029
:104F58007A1C0CD1DC692C40641B62425441B44277
:104F6800F6D00020E0BCBA46B146A846F0BDFCF732
:104F7800F9FC4B46C01AB84223D8002F21D043462B
:104F88001B681A685207E5D52A004021403A8A432F
:104F9800E0D008242100DA6911408A46144212D16F
:104FA8008022D96912011142D4D01A624046FFF713
:104FB800E7FA902320224146CA50424651460C3B0C
:104FC800D1540320CEE740461C62FFF7D9FA90235C
:104FD80042464146D45000220C3B0120CA54C1E746
:104FE8000022902330B50400C25083B0FCF7BAFC0D
:104FF800226805001168090710D4126852071CD4EA
:1050080020238822A3500432A35000230020E36603
:10501800236784230022E25403B030BD8021224B51
:1050280000220093890303002000FFF785FF002872
:1050380029D1226812685207E2D580211A4B002232
:10504800009320002B00C903FFF776FF0028D7D074
:10505800EFF31080012282F310882168134D0B684A
:105068002B400B6080F31088EFF3108082F31088D8
:1050780021688B6893438B6080F310888C231F32E0
:105088000320E250C5E7EFF31081012383F3108872
:105098008020226813688343136081F31088882373
:1050A80020220320E250B4E7FFFFFF01DFFEFFFFED
:1050B80010B5041E24D08823C358002B26D088237B
:1050C80024220121E250226813688B431360A36AEB
:1050D800002B17D12000FFF709FE012810D0236804
:1050E8000D495A6820000A402A215A609A688A4362
:1050F8009A601A6829390A431A60FFF771FF10BDD0
:105108000120FCE72000FFF7AFFEE3E78422835489
:10511800FCF70CFBD3E7C046FFB7FFFFF8B5130059
:105128005C2281650D0083522221902700228C2663
:10513800C25181515E310400405800280DD01E49EB
:105148008263C1621D492A0001631D4941632168C8
:105158002431FDF7C3F9002827D12369002B17D183
:10516800EFF31080012383F3108821688A681A43BB
:105178008A6080F31088EFF3108183F31088402051
:10518800226893680343936081F310880020F8BD78
:10519800EFF31081012383F310882268FF3310682E
:1051A8000343136081F31088DAE71023E3511033C7
:1051B8000120A351EBE7C046594C0008394C0008C0
:1051C8002948000803008C20185870B5202827D1DA
:1051D800002923D0002A21D080209C6840018442E5
:1051E80005D11869002802D10130CC0717D4002056
:1051F800D8661868406800020CD5EFF3108C0120BF
:1052080080F3108880201C68C0042568284320602B
:105218008CF310881800FFF781FF00E0012070BDB3
:105228000220FCE7F8B503680B4F9C689B680500F3
:105238005B0FF85C094EC000F15CFAF7EFFF6A23D8
:10524800E85223015B0FF85CF15CC000FAF7E6FF57
:105258006823E852F8BDC046C0660008B866000872
:105268007047C0467047C0467047C04670B5842432
:10527800035D012B12D0882524230126435103689E
:105288001A681968B143196005490A400021416646
:105298001A60202343510155002070BD0220FCE70D
:1052A800FFFFFFDF842370B5C35C04000A00012BF5
:1052B8001ED0882324210568C1502E682B68233905
:1052C8008B432B60AB68DB00D908436E1143A960A0
:1052D800002B0AD0FFF7A6FF882320222E60E25079
:1052E80000220020043BE25470BD024B8366F3E7C2
:1052F8000220F9E701000100842370B5C35C0400B3
:105308000A00012B1ED0882324210568C1502E686D
:105318002B6823398B432B60A9680B4B1940436ECC
:105328001143A960002B0AD0FFF77CFF88232022B5
:105338002E60E25000220020043BE25470BD034B73
:105348008366F3E70220F9E7FFFFFFF101000100A0
:10535800002370B54371FF330D00FF33510019402E
:10536800373B0270FF3B0A2204000548FEF726F887
:10537800FA222B1C5200954200D2131CE38070BD08
:1053880000010020F0B557464E46DE464546E0B5DA
:1053980087B00600171E059130D0194B00259B4693
:1053A8000F239A46102399460A23984608E0651960
:1053B800A619ADB20530B6B2FCF7DAFAAF421DD97C
:1053C80054464B4634401C1BA4B27B1BA34200DA54
:1053D8009CB243460293059B32005B190093A021BF
:1053E800012358460194FDF7EBFD0028DFD007B0F4
:1053F800F0BCBB46B246A946A046F0BD0020F6E781
:1054080000010020012310B5064C84B05B420293D2
:10541800019200910200A02120000233FDF7CCFE8A
:1054280004B010BD000100200A2310B50322A021FA
:105438000348FDF7C3FF431E9841C0B210BDC046E4
:105448000001002070B5002918D004006618012159
:105458000B480C4DB6B22378584008230A00024086
:105468004008002A01D0684080B2013BDBB2002B23
:10547800F4D10134A3B29E42EDD170BD0048FCE7DF
:10548800FFFF000001A0FFFFF0B5060087B00C0089
:105498001700FDF745F9730518D00025FF08361BDE
:1054A800002F04D10EE001350834AF420ADD22682E
:1054B800636801203119FDF781F90028F3D0012034
:1054C80007B0F0BDFDF7CAF90020F9E702230293FF
:1054D800F8231B06F318DB0A0493012301A902A889
:1054E8000593FDF7CDF90028D7D0E8E710B50400FB
:1054F800A02001222021C005FDF7ACFB22000A49AB
:105508000A48FFF78DF80A4C2000FDF703F9012837
:10551800FAD1043000F0CAFFA02000222021C005E3
:10552800FDF798FB10BDC0469006002058020020E9
:10553800A0010020F0B5DE4657464E464546E0B588
:10554800974E85B07388370058BA009383B29B464C
:10555800B388012298465BBA9BB29C46914C92490B
:10556800B01D08253B785C40130023406408002BDD
:1055780001D04C40A4B2013DEDB2002DF4D1013769
:10558800B842EED1230A9946884B894A5988E4B231
:105598005180197949B29180D98A002928D19580FA
:1055A8005979D180D9881181198951815989918175
:1055B8009989D181997B1182D97B187C0902014391
:1055C8005182598A9182998AD182D98A11835B8BB7
:1055D80053835B4663440E2B1BDCB379A34200D193
:1055E8006FE005B0F0BCBB46B246A946A046F0BD88
:1055F800D98A588B09B28246C8170918414089B21E
:105608005145CDD26B4909880629C9D99580DD82D3
:10561800C6E7FF23009A1B029A4219D180235B0038
:105628009845DED1B379A342DBD1F3794B45D8D184
:10563800614C624E03E0635D73550135EDB22000A5
:10564800FAF75AFD8542F6D3C0B2FFF74FFFC8E715
:10565800FD23009A1B029A42C3D1B379A342C0D159
:10566800F3794B45BDD1564B70781C886346534936
:105678003278000202430C71200A0E0001245B00FC
:10568800DBB21B040006134303430B60464D454B36
:105698004F1D327853400822200018405B0800282C
:1056A80001D06B409BB2013AD2B2002AF4D1013644
:1056B800BE42EED14B7107201B0A8B71FFF716FF14
:1056C8008FE7F3794B4500D08BE73C4933880B8053
:1056D80063465B008B704346002B59D05B46674698
:1056E8005800A44610188A4600223C00CB1C002112
:1056F800475E013239125F7097B219700230023377
:10570800A742F4D323004246644651469C460523EB
:10571800002A39D1DBB25A1E92B294461A000133DC
:10572800DBB20193931CDBB20293039565461E4FCF
:1057380094468B460120BA462A001A4B0D786B40D6
:10574800082507001F405B08002F02D057467B4002
:105758009BB2013DEDB2002DF3D1013A114D92B249
:105768000131AA42EAD1624659468B54019A1B0A72
:1057780002988B54039DFFF7B9FEFF23009A1B0282
:105788009A4200D14AE72CE763465B000333C1E73E
:1057980005230293013B0193023B03229C46C4E785
:1057A80090050020FFFF000001A0FFFF700500200A
:1057B80058030020740300201000002090060020E9
:1057C8000E000020F0B557464E464546DE46E0B589
:1057D800A34CA5B0638825000293A38801200393F6
:1057E800A379E61D9C4601939E4F9F4B66442A78F9
:1057F80053400822010019405B08002901D07B4072
:105808009BB2013AD2B2002AF4D10135B542EED1A9
:10581800019AA118FF22C8791A40904203D10A7A46
:105828001B0A9A4209D02378002B57D125B0F0BC27
:10583800BB46B246A946A046F0BD029A53BA9BB2EF
:1058480098468A4B99461B889A4698456BD9864B49
:105858009A42E8D104ABE11D802218009B4600F073
:1058680069FE21788023039A5B009A420ED1019B3E
:10587800022B0BD15B461B885BBA9BB2534500D108
:1058880095E07B4B00221A804B461A802378002B28
:10589800CCD0784B78481B7806000370102301247D
:1058A8004370029B6F4D4380039B871D83806E4B23
:1058B800327853400822210019405B08002901D0A2
:1058C8006B409BB2013AD2B2002AF4D10136BE42F3
:1058D800EED1C3800820FFF709FEA7E7654B6648AD
:1058E8001B78060003701023012443700F3B83705C
:1058F8005C4D5D4BC71C327853400822210019408B
:105908005B08002901D06B409BB2013AD2B2002A51
:10591800F4D10136B742EED1C3701B0A03710520DA
:10592800FFF7E4FD82E704AB18008022E11D9B46E7
:1059380000F000FE029B002B30D10133039AFF33A5
:105948009A421ED05346002BA0D18023039ADB0134
:105958009A429BD1019B802B98D1484B484D9C463D
:105968002888802259466044FFF78EFD00283ED1E2
:105978002B884A4680332B804B461B880133138083
:1059880084E7019B022B00D080E75B461B88384ADE
:105998005BBA138001234A46138077E7D0453DD090
:1059A800314B029A21789A4200D06FE75AE7344A7D
:1059B8002F4B10881A88904200D263E7002933D110
:1059C8002E4B304A1B68134080229205934200D028
:1059D8002CE72D48FCF7E0FB72B6284B2B4A936066
:1059E8002B4A12681B6883F3088890474EE7237890
:1059F800002B00D11AE71F4B1F4C1B780321237083
:105A08001023200063700F3BA370FFF71BFDE070AD
:105A1800000A20710520FFF769FD07E78023039A34
:105A2800DB019A42BCD195E7124B134D1B78032139
:105A38002B7010236B70113B6B80039B2800AB808D
:105A4800FFF700FDE8800820FFF750FD0B4B0D4ADB
:105A58001B68134080229205934200D016E7B8E7EE
:105A68009005002001A0FFFFFFFF00000C000020B0
:105A780054030020700500209006002000C800088C
:105A8800520300200000FE2F9C00002000ED00E0E3
:105A980004C80008F0B5DE4657464E464546E0B510
:105AA800C54D01202F00AB8885B09B466B88C34E3F
:105AB8000193C34BAC1D3A785340082201001940AA
:105AC8005B08002901D073409BB2013AD2B2002A88
:105AD800F4D10137A742EED1BA4928680860A888EE
:105AE800CB808880A979180ADBB2994202D1EB7978
:105AF800834206D005B0F0BCBB46B246A946A046D4
:105B0800F0BD5B465BBA98469EB2F02301991B0133
:105B180099421BD043461BB299468023019ADB0069
:105B28009A4228D1183B9E42E4D84346A64C03A982
:105B38002678E3805B46022205200B80F6B2FFF749
:105B480021FC002800D103E1E680D3E7731EF62B81
:105B5800D0D89D4CF6B2257802AB1A7101205E713F
:105B6800023203A9EDB22670FFF70CFC002800D121
:105B7800D6E02570BEE7A023019ADB009A425CD1EB
:105B8800924B934AF3189BB29342B3D88E4F3B89FA
:105B980079889BB29A464B469800484409B240001F
:105BA800FAF73CFB731F80B238810F2B00D9BEE097
:105BB80043463B813B89042B9CD93B89142B00D855
:105BC800BAE0C023019A1B019A4200D08DE0DC2381
:105BD800DC36B6B25B009E4200D98BE74B467A4F63
:105BE8003E8B36B2002B00D19EE07B8848461BB224
:105BF8009846FBF71DFA02000B0000207549FAF7DA
:105C0800F9FB040040460D00FBF712FA02000B00F6
:105C180020002900FAF708FFFBF7CEF900B2388315
:105C28003B8B03A95BBA02220F200B80FFF7AAFB6C
:105C380000283BD0B6B2BE825CE7C023019ADB00E5
:105C48009A4219D1FA23DB009C46FA236644B6B27D
:105C58001B019E4200D94DE743465B4F03A97C894F
:105C68007B815B46022209200B80A4B2FFF78AFBE6
:105C7800002855D07C813DE78023019A1B019A4278
:105C88006FD1032E00D935E700234F4C02AAA57B1C
:105C9800F6B2137156710320022203A9EDB2A6735E
:105CA800FFF770FB002801D0A57323E70820FFF752
:105CB8001DFC1FE7B023019A1B019A4200D080E720
:105CC800454B9E4200D915E73F4F03A9BB8A0222E4
:105CD8009BB299464346BB825B460D200B80FFF77B
:105CE80051FB00281CD04B46BB82D023019A1B01D4
:105CF8009A4200D0FEE6DC2E00D9FBE64346324C41
:105D080002AA658B63830023567113711120022246
:105D180003A9ADB2FFF736FB0028C7D06583E9E6D3
:105D28000830FFF7E3FBE5E601233B8378E73B898F
:105D3800042B00D8DEE640E75B4603A902220720D1
:105D48000B80FFF71FFB0028EAD053463B81CCE7C6
:105D58000830FFF7CBFB214AE38812689BB25363F4
:105D6800C8E6A023019A1B019A42A3D11A4B9E426E
:105D780000D9BFE6144F5A467B8A0B209BB29A463D
:105D880043467B8202AB9A8003A90222FFF7FAFA04
:105D980000280DD053467B82B023019A1B019A42FA
:105DA8001ED0C023019A1B019A4200D0A2E60EE73A
:105DB8000830FFF79BFB04E79005002001A0FFFFD8
:105DC800FFFF00009006002070050020E40C000092
:105DD800C819000000805B40DC0500005401002069
:105DE80043465A46BC8ABB8202AB9A800D200222E7
:105DF80003A9A4B2FFF7C6FA002800D156E7BC826F
:105E080078E6C04610B50F4B0F491A7809788A42D0
:105E180007D0002A04D15B78062B0FD0102B0AD0AC
:105E280010BD5B78062B09D0102B04D0032BF7D1BB
:105E3800FFF780FBF4E7FFF7C5FCF1E7FFF72AFE61
:105E4800EEE7C046900500207005002070B5284C8C
:105E580005002000FEF7C6FB012D3AD0022D35D0F3
:105E6800033D6B425D41234B6D421D4096239B01D0
:105E78009C466544204B0C2223600023200065606B
:105E8800A360E36023616261A361E36123626362EB
:105E9800A362FFF70DF9002827D100212000FFF7A2
:105EA80001FA00281ED100212000FFF725FA00285A
:105EB80015D12000FFF7DAF900280DD11021236849
:105EC8001A680A431A6050221A6270BDE1252D0231
:105ED800D0E79625ED01CDE7FBF7DEFAEEE7FBF715
:105EE800DBFAE6E7FBF7D8FADDE7FBF7D5FAD4E704
:105EF80058020020809C010000380140102170B534
:105F08004A4C86B0236801AD1A680A431A605022C9
:105F18001A6200F049FAFA213822C9004448FFF70A
:105F280017FAFFF781FA434E3000FEF7E1F8002137
:105F38003000FEF795F92000FEF7CAFB80223E49A3
:105F480052002000FFF73EF9FA223C493C48FCF792
:105F580085F8A02000222021C005FCF77BFE122234
:105F680029000020FFF74EFA00283FD16B78354C06
:105F780023702378FF2B3ED0EB78A373A37BFF2BF2
:105F880040D0A07BFFF762FFAB885BBAE380E28872
:105F98002D4B9A4239D0E38832689BB25363EB8821
:105FA8005BBA23812289284B9A4232D02B895BBA6B
:105FB80063816289244B9A422ED06B895BBA6382D3
:105FC800628A214B9A422AD0AB895BBAA382A28A01
:105FD8001D4B9A4226D0EB895BBA2383238B2B8AED
:105FE8005BBA6383628B184B9A4201D006B070BDCE
:105FF8003C236383FAE7FE3B2370EB78A373A37B10
:10600800FF2BBED10023A373BBE7AF239B00E38024
:10601800C1E70A232381C9E700236381CDE7282349
:106028006382D1E70023A382D5E7C0465802002047
:106038000C03002054010020900700207C0300205E
:106048009C00002070050020FFFF0000F8B5CE4638
:1060580004004746A020402180B5C005FCF7F4FDA8
:10606800774D80212870A020C005FCF7EDFD802C1D
:1060780007D0082C28D0734BDC60C0BCB946B046AA
:10608800F8BD0128F7D1FBF76DFC6F4F06003B68A0
:10609800C31A072B00D880E02B783E60012B00D173
:1060A80076E06A4A13780133DBB21370092BE2D920
:1060B800674B1978022900D883E0012065490870E8
:1060C800002111701970D6E70320634900F0C6F962
:1060D800A0200821C005FCF7B7FD0128CBD15F4BF4
:1060E8005F49604D18700B882A889B1A5E4A1BB25C
:1060F80093810B882E88578A1BB236B29B1BBB42F2
:1061080032DD0B881BB2002B5FDD00275748584E45
:10611800037837700133DBB298460370022B35D908
:10612800544E17714346FA2B01D9032303702B8869
:106138003380938A092B13D90B88908A1BB2DE17F8
:106148009B1973409BB283420AD22B88908A1BB258
:10615800DD175B196B409BB2834201D20023137198
:1061680053881BB20B8086E7414B0027984646466A
:106178001B780133DBB233703C4E3770012B05D9E5
:106188001071FA2B02D9032340460370394ECEE72B
:106198002F4A13780133137083E7FA21042089000A
:1061A80000F05CF9304B98465B79012B00D073E71F
:1061B800FA210220490000F051F9002342465371A8
:1061C8006AE7FF20234908707AE70B88294E9C4626
:1061D8000023F75E6346DB1B1BB293810B881BB25F
:1061E8009846538A9C464346DB1B634511DD0027CE
:1061F800BC461E4803780133DBB2984603701C4B3B
:106208001F0063463B704346022B90D963461371C7
:1062180088E7174B9C4667461B780133DBB23B7017
:1062280099460023114F3B704B46022B00D87EE75E
:106238001071FA2B00D87AE703236046037076E7DB
:1062480050030020001802404C030020480300209F
:106258004903002022000020881300008C0500203C
:1062680078030020760300207005002047030020F3
:10627800460300204403002010B5082800D010BDB4
:10628800A0200821C005FCF7DFFC002801D1044B41
:106298001870044B044A5B881BB21380EFE7C046B2
:1062A8008C050020700500207603002030B5354CA1
:1062B80089B02378FF2B40D0FFF720FE00236A46E1
:1062C80093810222402003A9FFF79CF80028F8D107
:1062D8006B469B892C4A5BBA013B9BB2934207D918
:1062E8002A4C2B4A2368134080229205934238D0C7
:1062F8006421002000F0B2F8264C002000F0C4F819
:1063080000280BD12378002BF7D0FFF77BFD002363
:106318000020237000F0B8F80028F3D080211E4830
:106328004900FCF79DFC80211B488900FCF798FC7C
:1063380020211948FCF794FCE4E71222FF2103A866
:1063480000F0CCF803A912220020FFF71BF8002266
:10635800002369460092019320000832FFF794F861
:10636800AAE70E4D2B68A342C2D972B60C48FBF7B8
:1063780013FF0C4B9C602B68226882F308889847AF
:10638800B6E7C04600900108FDFF000000C80008FD
:106398000000FE2F900800200004005004C80008E8
:1063A8009C00002000ED00E00022002110B5064C02
:1063B80053009B189B00E0180132416081604170D6
:1063C800E1540A2AF4D110BD980800201D4B30B5BD
:1063D8001A68002A04D01A68013A1A60002A2DD0D7
:1063E80000220125184C53009B189B00E1184868AF
:1063F80000280AD0486801384860002805D14D7047
:10640800E35C012B01D18B684B6001320A2AEAD187
:106418000E4B1A6801321A6019680D4A914201D16F
:1064280000221A60092000220A490B780133DBB2E6
:1064380098425241524213400B7030BD064B013214
:106448001A70CDE71409002098080020940800204D
:10645800FFFFFF7F910800201009002010B50928D0
:106468000FD8012484F310884300064A1B189B00A8
:10647800D0184160816000214170D45481F31088A4
:1064880010BDFEE798080020092808D84200121815
:10649800054B92009B185A78D0B2012A01D00020EF
:1064A800704700225A70FBE79808002000280ED099
:1064B80001280DD0012383F31088064B064A186083
:1064C8000023137083F310881378012BFCD17047D5
:1064D8000130EFE71409002010090020030082189A
:1064E800934200D1704719700133F9E770B500265F
:1064F8000C4C0D4D641BA410A64209D1002600F0D7
:1065080023F80A4C0A4D641BA410A64205D170BD9D
:10651800B300EB5898470136EEE7B300EB589847BD
:106528000136F2E7C8660008C8660008CC660008AD
:10653800C8660008002310B59A4200D110BDCC5C93
:10654800C4540133F8E70000F8B5C046F8BC08BCED
:106558009E467047F8B5C046F8BC08BC9E467047D2
:10656800E4040008D6040008B4040008E0040008A5
:10657800B4040008CA070008B4040008E0040008CE
:10658800D6040008D6040008CA070008E00400087A
:106598009C0400089C0400089C0400083C080008AF
:1065A80000000000000000000000000000000000E3
:1065B80001000000020000000300000004000000C9
:1065C80000000000000000000000000000000000C3
:1065D80000000000000000000000000000000000B3
:1065E8000100000002000000030000000400000099
:1065F8000600000007000000080000000900000075
:106608007A4100086A4100086A4100086A410008A6
:10661800CC4100086A4100086A4100086A41000844
:10662800E44100086A4100086A4100086A4100081C
:10663800FC4100086A4100086A4100086A410008F4
:1066480014420008B444000880440008804400084C
:1066580080440008DA4400088044000880440008A8
:10666800804400080445000880440008804400086D
:10667800804400082A450008804400088044000837
:1066880080440008544500088044000880440008FD
:10669800804400088A440008010002000400060043
:1066A80008000A000C0010002000400080000001D3
:1066B80008040204080101010101010307010000A7
:0466C800E1000008E5
:0466CC00B900000809
:1066D0000024F40001000000040000000100580242
:1066E0004443452D323430362D56362E305F4841E6
:0466F0004C00010059
:040000050800188D4A
:00000001FF
